** EXPERIMENTAL (HLL) ** Open Watcom Linker Version 1.6beta1 Limited Availability
Portions Copyright (c) 1985-2002 Sybase, Inc. All Rights Reserved.
Created on:       13/11/17 16:25:28
Warning! W1121: file U:/tmp\ldconv_zlibmodule_obj_1a8b52885a4f123668.obj(U:\DEV\python-2.7.5\Modules\zlibmodule.c): '_initzlib' has already been exported
Executable Image: build/lib.os2knix-2.7/zlib.pyd
creating an OS/2 EMX dynamic link library


                        +------------+
                        |   Groups   |
                        +------------+

Group                           Address              Size
=====                           =======              ====

CGROUP                          0001:00000000        0000f0f0
DGROUP                          0002:00000000        00001060



                        +--------------+
                        |   Segments   |
                        +--------------+

Segment                Class          Group          Address         Size
=======                =====          =====          =======         ====

TEXT32                 CODE           CGROUP         0001:00000000   0000f0f0
________TEXT           CODE           CGROUP         0001:0000f0f0   00000000
DATA32                 DATA           DGROUP         0002:00000000   00000fb0
SET1__os2dll           DATA           DGROUP         0002:00000fb0   00000004
SET2__os2dll           DATA           DGROUP         0002:00000fb4   00000000
SET3__os2dll           DATA           DGROUP         0002:00000fb4   00000004
SET1___CTOR_LIST__     DATA           DGROUP         0002:00000fb8   00000004
SET2___CTOR_LIST__     DATA           DGROUP         0002:00000fbc   00000000
SET3___CTOR_LIST__     DATA           DGROUP         0002:00000fbc   00000004
SET1___DTOR_LIST__     DATA           DGROUP         0002:00000fc0   00000004
SET2___DTOR_LIST__     DATA           DGROUP         0002:00000fc4   00000000
SET3___DTOR_LIST__     DATA           DGROUP         0002:00000fc4   00000004
SET1___crtinit1__      DATA           DGROUP         0002:00000fc8   00000004
SET2___crtinit1__      DATA           DGROUP         0002:00000fcc   00000000
SET3___crtinit1__      DATA           DGROUP         0002:00000fcc   00000004
SET1___crtexit1__      DATA           DGROUP         0002:00000fd0   00000004
SET2___crtexit1__      DATA           DGROUP         0002:00000fd4   00000000
SET3___crtexit1__      DATA           DGROUP         0002:00000fd4   00000004
SET1___eh_frame__      DATA           DGROUP         0002:00000fd8   00000004
SET2___eh_frame__      DATA           DGROUP         0002:00000fdc   0000000c
SET3___eh_frame__      DATA           DGROUP         0002:00000fe8   00000004
SET1___eh_init__       DATA           DGROUP         0002:00000fec   00000004
SET2___eh_init__       DATA           DGROUP         0002:00000ff0   00000004
SET3___eh_init__       DATA           DGROUP         0002:00000ff4   00000004
SET1___eh_term__       DATA           DGROUP         0002:00000ff8   00000004
SET2___eh_term__       DATA           DGROUP         0002:00000ffc   00000004
SET3___eh_term__       DATA           DGROUP         0002:00001000   00000004
SET1___fork_parent1__  DATA           DGROUP         0002:00001004   00000004
SET2___fork_parent1__  DATA           DGROUP         0002:00001008   00000000
SET3___fork_parent1__  DATA           DGROUP         0002:00001008   00000004
SET1___fork_child1__   DATA           DGROUP         0002:0000100c   00000004
SET2___fork_child1__   DATA           DGROUP         0002:00001010   00000000
SET3___fork_child1__   DATA           DGROUP         0002:00001010   00000004
________DATA           DATA           DGROUP         0002:00001020   00000000
BSS32                  BSS            DGROUP         0002:00001020   00000040
c_common               BSS            DGROUP         0002:00001060   00000000
________BSS            BSS            DGROUP         0002:00001060   00000000


                        +----------------+
                        |   Memory Map   |
                        +----------------+

* = unreferenced symbol
+ = symbol only referenced locally

Address        Symbol
=======        ======

Module: U:\usr\lib\dll0hi.obj({standard input})
0001:00000000* __text
0002:00000000* __data
0002:00000000* ___data_start
0002:00001020* ___bss_start
0002:00000fb0+ __os2dll
0002:00000fb8  ___CTOR_LIST__
0002:00000fc0  ___DTOR_LIST__
0002:00000fc8* ___crtinit1__
0002:00000fd0* ___crtexit1__
0002:00000fd8  ___eh_frame__
0002:00000fec  ___eh_init__
0002:00000ff8  ___eh_term__
0002:00001004+ ___fork_parent1__
0002:0000100c+ ___fork_child1__
Module: U:/tmp\ldconv_zlibmodule_obj_1a8b52885a4f123668.obj(U:\DEV\python-2.7.5\Modules\zlibmodule.c)
0001:000022d0  _initzlib
Module: U:\usr\local473\lib\libc_dll.lib(dllinit.obj)
0001:00002550  _DLL_InitTerm
Module: U:\usr\lib\libend.lib(src/libend/386/endlink386.asm)
0002:00001060  _end
0002:00001020  _edata
Module: U:\usr\lib\libend.lib(src/libend/386/end.asm)
0001:0000f0f0* _etext
0001:0000f0f0* __etext
0000:00000000  WEAK$ZERO
0002:00001060  __end
0002:00001020  __edata
Module: U:\extras\lib\libz.lib(crc32.obj)
0001:0000280c* _get_crc_table
0001:00002818  _crc32
0001:00002b00* _crc32_combine
0001:00002b24* _crc32_combine64
Module: U:\extras\lib\libz.lib(adler32.obj)
0001:00004b50  _adler32
0001:00004dc0* _adler32_combine
0001:00004e68* _adler32_combine64
Module: U:\extras\lib\libz.lib(inflate.obj)
0001:00005064* _inflateReset
0001:00005110* _inflateReset2
0001:00005254  _inflateInit2_
0001:00005314* _inflateInit_
0001:000053d8* _inflatePrime
0001:00005610  _inflate
0001:00007498  _inflateEnd
0001:000074f4* _inflateSetDictionary
0001:000075e0* _inflateGetHeader
0001:00007610* _inflateSync
0001:0000780c* _inflateSyncPoint
0001:00007840  _inflateCopy
0001:000079a8* _inflateUndermine
0001:000079d4* _inflateMark
Module: U:\extras\lib\libz.lib(deflate.obj)
0001:000092e8* _deflateSetDictionary
0001:00009414* _deflateReset
0001:00009580* _deflateSetHeader
0001:000095ac* _deflatePrime
0001:000095e4* _deflateTune
0001:00009624* _deflateBound
0001:00009750  _deflate
0001:0000a69c* _deflateParams
0001:0000a790  _deflateEnd
0001:0000a860  _deflateInit2_
0001:0000aae4  _deflateInit_
0001:0000ace0  _deflateCopy
0001:0000aeb0* _deflate_copyright
Module: U:\tmp\ldconv_libgcc_so_d_a_1a8b52885a4f12bf20.lib(emx-ctordtor.obj)
0001:0000af80  ___ctordtorInit
0001:0000afb4  ___ctordtorTerm
Module: U:\tmp\ldconv_libgcc_a_1a8b52885a4f12bf20.lib(_moddi3.obj)
0001:0000aff0  ___moddi3
Module: U:\extras\lib\libz.lib(zutil.obj)
0001:0000b178* _zlibVersion
0001:0000b184* _zlibCompileFlags
0001:0000b190* _zError
0001:0000b250  _z_errmsg
0001:0000b1a4  _zcalloc
0001:0000b1bc  _zcfree
Module: U:\extras\lib\libz.lib(inftrees.obj)
0001:0000b280  _inflate_table
0001:0000bad0* _inflate_copyright
Module: U:\extras\lib\libz.lib(inffast.obj)
0001:0000bc50  _inflate_fast
Module: U:\extras\lib\libz.lib(trees.obj)
0001:0000e810  __length_code
0001:0000e610  __dist_code
0001:0000d6f8  __tr_init
0001:0000d7d0  __tr_stored_block
0001:0000d87c  __tr_align
0001:0000dbac  __tr_flush_block
0001:0000e578* __tr_tally
Module: U:\tmp\ldconv_libgcc_so_d_a_1a8b52885a4f12bf20.lib(emx-eh.obj)
0001:0000f080  ___ehInit
0001:0000f0b6* ___ehTerm


                        +----------------------+
                        |   Imported Symbols   |
                        +----------------------+

Symbol                              Module
======                              ======

___libc_ForkRegisterModule          libc065
___init_dll                         libc065
___libc_Back_termDll                libc065
___libc_ForkDeregisterModule        libc065
__atfork_callback                   libc065
_PyArg_ParseTuple                   python27
_PyInt_FromLong                     python27
_Py_FindMethod                      python27
_PyEval_SaveThread                  python27
_PyThread_acquire_lock              python27
_PyEval_RestoreThread               python27
_PyThread_release_lock              python27
_PyString_FromStringAndSize         python27
_PyErr_NoMemory                     python27
_PyObject_Free                      python27
__PyString_Resize                   python27
_PyErr_Format                       python27
_PyExc_ValueError                   python27
_PyErr_SetString                    python27
__PyObject_New                      python27
_PyString_FromString                python27
_PyExc_MemoryError                  python27
_PyType_Type                        python27
_Py_InitModule4                     python27
_PyErr_NewException                 python27
_PyModule_AddObject                 python27
_PyModule_AddIntConstant            python27
_PyModule_AddStringConstant         python27
_PyThread_allocate_lock             python27
__CRT_init                          libc065
__CRT_term                          libc065
__std_memcpy                        libc065
__std_malloc                        libc065
__std_free                          libc065
___ctordtorInit1                    libc065
___ctordtorTerm1                    libc065
___register_frame_table             gcc473
___deregister_frame                 gcc473


                        +--------------------+
                        |   Libraries Used   |
                        +--------------------+

U:\extras\lib\libz.lib
U:\tmp\ldconv_python2_7_dll_a_1a8b52885a4f128488.lib
U:\tmp\ldconv_libgcc_a_1a8b52885a4f12bf20.lib
U:\tmp\ldconv_libgcc_so_d_a_1a8b52885a4f12bf20.lib
U:\usr\lib\libc_alias.lib
U:\usr\local473\lib\libc_dll.lib
U:\usr\lib\libend.lib


                        +-----------------------+
                        |   Linker Statistics   |
                        +-----------------------+

Stack size:  0000 (0.)
Memory size:  00010150 (65872.)
Link time: 00:00.06
